:020000040000FA
:04000000EE303A287C
:08000800A000030EA100831209
:1000100005191028831601178312B23081002B288E
:1000200083160113831203140B190310A80DA90DD5
:10003000AA0DAB0DAC0DAC16FF302C02031D2B2806
:10004000FA302B02031D2B2831152A08AF0029088E
:10005000AE002808AD008B100B11210E8300A00EFE
:04006000200E090065
:0C007400203084008001840A80300402E7
:10008000031C3C281230B000092283160C30850571
:1000900087018312850187010730990000309A009B
:1000A000103083168E008312603083168F00831207
:1000B0000030831691009F008312C83083168100A0
:1000C000831231309000003083168C008312103080
:1000D0008B00792381018E018F010B118B100B1086
:1000E0008C018B17812031198420B30B7F280310DA
:1000F00085190314B90DF030390203195721E02393
:10010000722864003210080031110130B7008B13DF
:1001100020303707371A313E83169B001C141A080B
:100120008312A40010303707371A313E83169B0024
:100130001C141A088312A300A6000230A606003081
:100140003707371A313E83169B001C141A08831296
:10015000A200A7000130A7068B17321CB528220980
:100160000339A200A309A409A50924082F02031D2D
:10017000512923082E02031D512922082D02031D97
:10018000512901303702031DCA283D18CA283D14E1
:100190003E14242202303702031DD328BD18D32871
:1001A000BD143E14352203303702031DDC283D19EF
:1001B000DC283D153E14462204303702031DE52895
:1001C000BD19E528BD153E14572205303702031D21
:1001D000EE283D1AEE283D163E14682206303702FE
:1001E000031DF728BD1AF728BD163E1478220730E4
:1001F0003702031D00293D1B00293D173E148822AC
:1002000008303702031D0929BD1B0929BD173E14FB
:10021000982209303702031D12295D1812295D1436
:100220003E14A8220A303702031D1B29DD181B29A2
:10023000DD143E14B8220B303702031D24295D194A
:1002400024295D153E14C8220C303702031D2D29C8
:10025000DD192D29DD153E14D8220D303702031D7E
:1002600036295D1A36295D163E14E8220E30370213
:10027000031D3F29DD1A3F29DD163E14F8220F30F9
:100280003702031D48295D1B48295D173E140823CA
:1002900010303702031D5129DD1B5129DD173E1493
:1002A0001823B70A0F3037020318080087280130D7
:1002B000B600B300B400B500B70085018701B113E3
:1002C0008120B30BAF29031085190314B90DF03049
:1002D00039020319DC29B40BAF29013037020319A5
:1002E00029230230370203192E2303303702031962
:1002F000332304303702031938230530370203193A
:100300003D23063037020319422307303702031911
:1003100047230830370203194C23093037020319E9
:1003200051230A303702031956230B3037020319C1
:100330005B230C303702031960230D303702031999
:1003400065230E30370203196A230F303702031971
:100350006F2310303702031974239630B400311D17
:1003600060293111321CB9292D090339AD00AE09BC
:10037000AF092F1C60298E018F010C1C60290C1005
:100380002E1E60298B1320303707371A313EBB00F1
:100390002F08BA00F42110303707371A313EBB005E
:1003A0002E08BA00F42100303707371A313EBB005F
:1003B0002D08BA00F4218B1785018701B70AB60111
:1003C0000F303702031C6029792308003E1C080007
:1003D0003E101030BB003D08BA00F4213030BB00A5
:1003E0005D08BA00F42108008B133A0883161C1527
:1003F0009A0083123B0883169B0055309D00AA305B
:100400009D009C1464009C18022A1C1183128B17F7
:100410000800831610309B001C141A088312BD00BC
:10042000831630309B001C141A088312DD00FF3045
:10043000C800CA15CB15CC15CD15CE15CF15D015C6
:10044000D115D215D31508000130BD050030DD05EA
:100450005F140530C405C0000030C2004030C5053F
:10046000C1004030C3005E1008000230BD050030FE
:10047000DD055F143530C405C0000030C2004030D7
:10048000C505C1004030C3005E1008000430BD0542
:100490000030DD055F140530C405C0000430C20023
:1004A0004030C505C1004030C3005E100800083070
:1004B000BD050030DD055F144830C405C0000030C4
:1004C000C2008030C505C1008030C3005E10080046
:1004D0001030BD050030DD055F14CA30C405C00012
:1004E0008030C2008030C505C1008030C3000800E4
:1004F0002030BD050030DD055F142930C405C00083
:100500000030C2004030C505C1004030C3000800C3
:100510004030BD050030DD055F141930C405C00052
:100520000030C2004030C505C1004030C3000800A3
:100530008030BD050030DD055F14AA30C405C00061
:100540008030C2008030C505C1008030C300080083
:100550000030BD050130DD055F149A30C405C000D0
:100560008030C2008030C505C1008030C300080063
:100570000030BD050230DD055F143930C405C00010
:100580000030C2004030C505C1004030C300080043
:100590000030BD050430DD055F14B230C405C00075
:1005A0008030C2008030C505C1008030C300080023
:1005B0000030BD050830DD055F142230C405C000E1
:1005C0000230C2004030C505C1004030C300080001
:1005D0000030BD051030DD055F143230C405C000A9
:1005E0001230C2004030C505C1004030C3000800D1
:1005F0000030BD052030DD055F140830C405C000A3
:100600000030C200C030C505C100C030C3000800C2
:100610000030BD054030DD055F140030C405C0006A
:100620000030C2000030C505C1000030C300080022
:100630000030BD058030DD055F140030C405C0000A
:100640000030C2000030C505C1000030C300080002
:100650000800113085061030870608001130850625
:10066000163087060800113085061030870608000E
:1006700002308506093087060800223085062930B9
:1006800087060800123085061430870608001230ED
:100690008506123087060800223085062C30870632
:1006A0000800223085062A308706080012308506A9
:1006B000163087060800203085062E308706080091
:1006C0002030850614308706080020308506163055
:1006D00087060800023085061830870608000030BB
:1006E0008506003087060800003085060030870642
:1006F00008003D182422BD1835223D194622BD1997
:1007000057223D1A6822BD1A78223D1B8822BD1B44
:1007100098225D18A822DD18B8225D19C822DD19BB
:10072000D8225D1AE822DD1AF8225D1B0823DD1BA2
:1007300018230800B601B301B4013C1CA22BBC0174
:10074000BC14A42BBC013C143C08B6006400A82BCC
:10075000A92BAA2BAB2BAC2BFF30B41B8500B41FED
:100760008501B30BA62BB40BA62B0310B60CB60851
:10077000031DA62B0030BB003C08BA00F421080082
:1007800005125C180516DC1C8512DC1885165C1D2C
:1007900005105C190514DC1D8510DC1985145C1E20
:1007A00087105C1A8714DC1E0711DC1A07155C1F02
:1007B00007105C1B0714DC1F8712DC1B8716080060
:1007C0008F08031908008F0178308E00C80FA02E03
:1007D000C80A5F1CF42B4208C6054308C705460833
:1007E000C2064708C3065F104208430403196B2C76
:1007F00046084704031D032C4208C600C2014308F3
:10080000C700C3016B2C46184A08C6184B08461986
:100810004C08C6194D08461A4E08C61A4F08461B02
:100820005008C61B5108471B5208C71B5308E0005D
:10083000421C202C4A086002031942100319461476
:10084000C21C282C4B0860020319C2100319C614DD
:10085000421D312C4C086002031D312C42114615FB
:100860004415C21D392C4D0860020319C211031929
:10087000C615421E412C4E0860020319421203198C
:100880004616C21E492C4F0860020319C2120319F2
:10089000C616421F512C5008600203194213031957
:1008A0004617C21F592C510860020319C2130319BD
:1008B000C617471B632C431F632C520860020319A1
:1008C000431303194717C31F6B2C53086002031906
:1008D000C3130319C717DE19942C441C942C461C0F
:1008E000852CCA1C762CCA014A15A22C4A1D7B2CC9
:1008F000CA01CA15A22CCA1D802CCA014A16A22CF4
:100900004A1EA22CCA01CA14A22C4A1D8A2CCA0152
:100910004A16A22CCA1D8F2CCA014A16A22C4A1EA6
:10092000A22CCA01CA14A22CCA1C992CCA014A15AD
:10093000A22C4A1D9E2CCA01CA15A22C4A1EA22C0A
:10094000CA014A15DE19CB2CC41CCB2CC61CBC2CEE
:10095000CB1CAD2CCB014B15D92C4B1DB22CCB0194
:10096000CB15D92CCB1DB72CCB014B16D92C4B1E3C
:10097000D92CCB01CB14D92C4B1DC12CCB014B1640
:10098000D92CCB1DC62CCB014B16D92C4B1ED92CE8
:10099000CB01CB14D92CCB1CD02CCB014B15D92C93
:1009A0004B1DD52CCB01CB15D92C4B1ED92CCB01F3
:1009B0004B15DE19022D441D022D461DF32CCC1CB7
:1009C000E42CCC014C15102D4C1DE92CCC01CC1580
:1009D000102DCC1DEE2CCC014C16102D4C1E102DC4
:1009E000CC01CC14102D4C1DF82CCC014C16102D24
:1009F000CC1DFD2CCC014C16102D4C1E102DCC0105
:100A0000CC14102DCC1C072DCC014C15102D4C1DD9
:100A10000C2DCC01CC15102D4C1E102DCC014C15DD
:100A2000DE193A2DC41D3A2DC61D2B2DCD1C1C2DB3
:100A3000CD014D155E13482D4D1D212DCD01CD1538
:100A4000482DCD1D262DCD014D16482D4D1E482D6E
:100A5000CD01CD14482D4D1D302DCD014D16482D05
:100A6000CD1D352DCD014D16482D4D1E482DCD01E6
:100A7000CD14482DCD1C3F2DCD014D15482D4D1DBC
:100A8000442DCD01CD15482D4D1E482DCD014D15C0
:100A9000DE19732D5E1B732D441E732D461E642DAF
:100AA000CE1C552DCE014E15812D4E1D5A2DCE0139
:100AB000CE15812DCE1D5F2DCE014E16812D4E1EE1
:100AC000812DCE01CE14812D4E1D692DCE014E16E5
:100AD000812DCE1D6E2DCE014E16812D4E1E812DE7
:100AE000CE01CE14812DCE1C782DCE014E15812D38
:100AF0004E1D7D2DCE01CE15812D4E1E812DCE0198
:100B00004E15DE19AA2DC41EAA2DC61E9B2DCF1C64
:100B10008C2DCF014F15B82D4F1D912DCF01CF1525
:100B2000B82DCF1D962DCF014F16B82D4F1EB82DC5
:100B3000CF01CF14B82D4F1DA02DCF014F16B82DCA
:100B4000CF1DA52DCF014F16B82D4F1EB82DCF01AB
:100B5000CF14B82DCF1CAF2DCF014F15B82D4F1D81
:100B6000B42DCF01CF15B82D4F1EB82DCF014F1585
:100B7000DE19E12D441FE12D461FD22DD01CC32DBF
:100B8000D0015015EF2D501DC82DD001D015EF2DDF
:100B9000D01DCD2DD0015016EF2D501EEF2DD001C0
:100BA000D014EF2D501DD72DD0015016EF2DD01D94
:100BB000DC2DD0015016EF2D501EEF2DD001D0149A
:100BC000EF2DD01CE62DD0015015EF2D501DEB2D33
:100BD000D001D015EF2D501EEF2DD0015015DE198C
:100BE000182EC41F182EC61F092ED11CFA2DD10194
:100BF0005115262E511DFF2DD101D115262ED11DA7
:100C0000042ED1015116262E511E262ED101D114AB
:100C1000262E511D0E2ED1015116262ED11D132E1A
:100C2000D1015116262E511E262ED101D114262E69
:100C3000D11C1D2ED1015115262E511D222ED10160
:100C4000D115262E511E262ED1015115DE19502EFA
:100C5000451F502E471F412ED21C322ED201521555
:100C6000DE135E2E521D372ED201D2155E2ED21DFE
:100C70003C2ED20152165E2E521E5E2ED201D2148E
:100C80005E2E521D462ED20152165E2ED21D4B2EC6
:100C9000D20152165E2E521E5E2ED201D2145E2E4C
:100CA000D21C552ED20152155E2E521D5A2ED20143
:100CB000D2155E2E521E5E2ED2015215DE19892EDD
:100CC000DE1B892EC51F892EC71F7A2ED31C6B2EC3
:100CD000D3015315972E531D702ED301D315972E84
:100CE000D31D752ED3015316972E531E972ED30165
:100CF000D314972E531D7F2ED3015316972ED31D39
:100D0000842ED3015316972E531E972ED301D3143E
:100D1000972ED31C8E2ED3015315972E531D932E31
:100D2000D301D315972E531E972ED3015315E621C9
:100D30004008C4004108C5005E18DE145E1CDE10C9
:100D40004808C9000C304A05031D05120C304B053C
:100D5000031D85120C304C05031D05100C304D058C
:100D6000031D85100C304E05031D87100C304F05F8
:100D7000031D07110C305005031D07100C305105E1
:100D8000031D87120C305205031D07120C3053054A
:100D9000031D871149080E020318FA2E12304A0566
:100DA000031D051612304B05031D851612304C0528
:100DB000031D051412304D05031D851412304E0518
:100DC000031D871412304F05031D071512305005FF
:100DD000031D071412305105031D871612305205EA
:100DE000031D071612305305031D8715FF304802F7
:100DF000031908008F08031D0800812049080E020E
:100E0000031CFA2E18304A05031D051206304A0548
:100E1000031D051618304B05031D851206304B05C2
:100E2000031D851618304C05031D051006304C05B2
:100E3000031D051418304D05031D851006304D05A2
:100E4000031D851418304E05031D871006304E050E
:100E5000031D871418304F05031D071106304F0579
:100E6000031D071518305005031D071006305005E7
:100E7000031D071418305105031D87120630510554
:100E8000031D871618305205031D07120630520540
:100E9000031D071618305305031D8711063053052F
:060EA000031D8715080088
:084000000E0003000500090099
:02400E00CC33B1
:10420000010078007A007C007E007B0079007F004E
:104210007D007A0078007E007C007D007F007900C0
:104220000200F200F600FA00FE00F200F600FA00CA
:10423000FE00F200F600FA00FE00F200F600FA00BE
:10424000FF00050005000500050009000900090040
:1042500009000D000D000D000D00110011001100EE
:104260000100FF00FF00FF00FF00FF00FF00FF0054
:10427000FF00FF00FF00FF00FF00FF00FF00FF0046
:10428000FF007B00FF00FF00FF00FF00FF00FF00BA
:10429000FF00FF00FF00FF00FF00FF00FF00FF0026
:1042A000FF00FE00FF00FF00FF00FF00FF00FF0017
:1042B000FF00FF00FF00FF00FF00FF00FF00FF0006
:1042C000FF001100FF00FF00FF00FF00FF00FF00E4
:1042D000FF00FF00FF00FF00FF00FF00FF00FF00E6
:1042E000FF00FF00FF00FF00FF00FF00FF00FF00D6
:1042F000FF00FF00FF00FF00FF00FF00FF00DD00E8
:00000001FF
